:1000000012C02CC02BC02AC029C028C027C026C0BF
:1000100025C02BC123C0E9C021C020C085C11EC09E
:100020001DC01CC01BC011241FBECFE5D4E0DEBF25
:10003000CDBF11E0A0E6B0E0E2ECFDE002C005902B
:100040000D92A23FB107D9F712E0A2EFB1E001C0D3
:100050001D92AD38B107E1F713D0B1C6D1CF9C01E5
:10006000E199FECF3FBB2EBBE09A8DB3089580E8A7
:1000700081BB80E187BB88E288BB82E082BB0895B8
:1000800080E881BB80E187BB88E288BB82E082BBDD
:10009000E7D08AD045D1E199FECF84E090E09FBBC4
:1000A0008EBBE09A8DB381BF80E090E06FE270E09C
:1000B000C4D4909358028093570282E090E06FE29C
:1000C00070E0BBD490935A028093590229E72093A1
:1000D0002C028091590290915A02C29711F42093F8
:1000E0002C028091590290915A028436910519F49C
:1000F00082EF80932C028091590290915A028B34A6
:10010000910519F482EA80932C0297987894609173
:10011000590270915A0285E090E049E150E0C6D260
:1001200085E58093450285E490E0909347028093B3
:10013000460285E690E090934A02809349028EEF52
:1001400090E090934C0280934B028091FC0187B920
:100150008FEC86B98091F3018130F9F41092F301AC
:100160009091FB018091600020E030E0803F11F031
:1001700021E030E0892F90E028233923232B09F058
:100180000AD32FD480E090E053D181E090E050D1A9
:100190008091F901863009F4EBD28091F40181302D
:1001A000C9F61092F401D6CF10BC83E389B910BC14
:1001B0001BB884E98AB98EEB80BD08955D9BFECFA4
:1001C0008CB90895662359F020E0FC01E20FF11D7F
:1001D000E0815D9BFECFECB92F5F6217B0F7089509
:1001E0005D9BFECF8EE38CB908951F920F920FB6E0
:1001F0000F9211242F938F939F938AB12CB19091DA
:10020000FA01913049F4919A209360008091600046
:10021000803F11F49093FB012F3F19F481E080930C
:10022000FA019F918F912F910F900FBE0F901F9009
:100230001895DC010D900020E9F71197A81BB90B68
:1002400020E030E009C0FC01E20FF31FE0815D9B7C
:10025000FECFECB92F5F3F4F2A173B07A0F308955D
:1002600082E083BF81E089BF08951F920F920FB68D
:100270000F9211248F939F93809106028F5F80933A
:1002800006028150843029F481E08093F7011092B6
:10029000060280915B028F5F80935B0280915B021C
:1002A0008732B9F591E09093F50110925B0280914D
:1002B00005028F5F8093050280910502853021F44D
:1002C000109205029093F601809103028F5F809354
:1002D000030280910302843639F41092030281E014
:1002E0008093F2018093F40180910302823319F428
:1002F00081E08093F401809104028F5F8093040277
:10030000809104028A3029F41092040281E08093E3
:10031000F3019F918F910F900FBE0F901F90189532
:1003200017B888E886B908951F920F920FB60F92FA
:1003300011241F932F933F934F935F936F937F935A
:100340008F939F93AF93BF93EF93FF9316B88091D2
:10035000FC01882309F040C0E091F101F0E084B194
:1003600095B1EE0FFF1FE45AFD4F91838083E0911A
:10037000F101F0E0EE0FFF1FE45AFD4F8081918103
:1003800090936A0280936902E091F101F0E0EE0F30
:10039000FF1FE45AFD4F80819181209157023091D7
:1003A0005802821B930B91838083E091F101F0E06E
:1003B000EE0FFF1FE45AFD4F8081918197FF09C026
:1003C000E091F101F0E0EE0FFF1FE45AFD4F1182C2
:1003D000108281E08093FE0181E0809307021091FA
:1003E000FC01113099F464B175B1882777FD8095CF
:1003F000982FE9D32DEC3CEC4CE950E449D3B0D331
:1004000070932B0260932A021093FD01FF91EF91EC
:10041000BF91AF919F918F917F916F915F914F911C
:100420003F912F911F910F900FBE0F901F90189525
:10043000AF92BF92CF92DF92EF92FF920F931F93F2
:100440008091FC01882319F08FC01092FE018091E9
:10045000FE018823D1F38091F1018F5F8093F10138
:100460008091F101853008F47FC01092F101EE24F3
:10047000FF24870140E050E0FA01EE0FFF1FE45A2D
:10048000FD4F2081318180912C0290E0BC01269F9C
:10049000C001279F900D369F900D1124AA2797FD2C
:1004A000A095BA2FE80EF91E0A1F1B1F4F5F5F4F62
:1004B0004530510509F7C801B70125E030E040E0BB
:1004C00050E02CD4D22EC32EB42EA52E809108023B
:1004D00090910902A0910A02B0910B02E80EF91E58
:1004E0000A1F1B1FE0920802F092090200930A0201
:1004F00010930B02E0900802F090090200910A02AA
:1005000010910B0285E580934502622F732F842F93
:10051000952F24E630E040E050E000D430935402C0
:10052000209353026D2D7C2D8B2D9A2D28EE33E0D8
:1005300040E050E0F3D324E630E040E050E0EED37A
:100540002093480285E690E090934A028093490206
:10055000C801B70120EA3CE840E050E0DFD3309327
:100560004C0220934B027BD08091FC01813081F4BE
:100570008091FD018823E1F31092FD018091F90142
:10058000823009F440D08091F901833009F43BD0E6
:100590008091FC018F5F8093FC018091FC0182308F
:1005A00011F41092FC018091FC0187B98FEC86B99F
:1005B0001F910F91FF90EF90DF90CF90BF90AF9081
:1005C00008959C01E199FECF3FBB2EBB6DBB0FB6DA
:1005D000F894E29AE19A0FBE0895609157027091E3
:1005E000580280E090E041EE52E03DD208959C0137
:1005F000E199FECF3FBB2EBB6DBB0FB6F894E29ADC
:10060000E19A0FBE089520912A0230912B02822F89
:100610006AE065D364D3382F5CE25093C400822F24
:100620005ED3292F205D2093C50059D3905D909310
:10063000C3005093EC002093ED009093EB00332324
:1006400011F480E202C0832F805D8093C20080930A
:10065000EA0086E58093C6008093EE00089520911D
:10066000530230915402C9016AE070E044D3462F2E
:10067000862F6AE034D3382F8CE28093CD00822F0E
:100680002ED3905D9093CE00842F29D3905D9093CC
:10069000CC00332321F480E28093CB0003C0305D93
:1006A0003093CB0081E48093CF000895CF92DF9206
:1006B000EF92FF920F931F93CF93DF93FC017B0187
:1006C0006A0177FD02C000E005C0F094E194F108F2
:1006D000F39401E0C70164E670E00DD3482F192FB1
:1006E0006AE070E008D3805D28E230E0E29FE0013C
:1006F000E39FD00DF29FD00D1124FE01EC0DFD1DE6
:10070000EF59FF4F8083960121503040842F912F65
:100710006AE070E0F0D2605DFE01E20FF31FEF5976
:10072000FF4F608321503040C70164E670E0E3D2A0
:10073000605DFE01E20FF31FEF59FF4F6083F90187
:100740003197002331F0EC0FFD1FEF59FF4F8DE281
:1007500005C0EC0FFD1FEF59FF4F80E28083DF9152
:10076000CF911F910F91FF90EF90DF90CF90089560
:100770006091690270916A0286E090E044E150E085
:1007800095DF609157027091580286E090E04BE14E
:1007900050E08CDF08958091F901833009F43FC067
:1007A000843028F4813099F0823048F509C08530D2
:1007B00009F450C08530D0F1863009F011C1DBC09A
:1007C00080916000803B09F00BC181E03EC08091C8
:1007D0006000803D21F41092F9011092FB0180919C
:1007E0006000803B29F482E08093F9011092FB01C4
:1007F00080916000803E09F0F3C084E026C08091C3
:100800006000803D29F481E08093F9011092FB01A2
:1008100080916000803B09F0E3C083E016C08091C6
:100820006000803D09F0DCC082E00FC08091600074
:10083000803729F481E08093F9011092FB018091C7
:100840006000803B09F0CCC085E08093F9011092F4
:10085000FB01089580916000803789F580915902ED
:1008600090915A028B34910571F08436910519F0FC
:10087000C297D1F410C08BE490E090935A02809319
:10088000590289E70FC082E390E090935A02809367
:1008900059028CE807C084E690E090935A02809356
:1008A000590288EC80932C021092FB01609159024E
:1008B00070915A0285E090E049E150E0F7DE8091C6
:1008C0006000803E89F58091590290915A028B34E4
:1008D000910571F08436910519F0C297D1F410C0DA
:1008E00082E390E090935A02809359028AE70FC006
:1008F00084E690E090935A028093590282EF07C0F9
:100900008BE490E090935A028093590282EA80939C
:100910002C021092FB016091590270915A0285E0FD
:1009200090E049E150E0C2DE80916000803D71F4CA
:1009300084E08093F9011092FB016091590270915B
:100940005A0282E090E047EF52E08DD08091600043
:10095000803B09F045C00CDF86E08093F9011092DE
:10096000FB016091590270915A0282E090E047EFDA
:1009700052E079D0089582B3805882BB80916000A4
:10098000803761F4809157029091580201979093BB
:10099000580280935702ECDE1092FB0180916000B8
:1009A000803E61F480915702909158020196909395
:1009B000580280935702DCDE1092FB0180916000A8
:1009C000803D71F4609157027091580280E090E090
:1009D00047EF52E048D085E08093F9011092FB0187
:1009E00008950F931F93CF93DF938CE98AB95098A2
:1009F0008EEFE4DBC0E0D0E008E210E0509A809196
:100A0000F90190E0809FF001819FF00D909FF00D23
:100A10001124EC0FFD1FEF59FF4F8081CFDB219692
:100A2000C032D10559F750988FEFC8DB9198539891
:100A3000DF91CF911F910F910895DF92EF92FF9276
:100A40000F931F937B018C01FB010995D82EC801E0
:100A50000196F7010995982F8D2D1F910F91FF9009
:100A6000EF90DF900895DF92EF92FF920F931F9324
:100A7000D72E7A018C01FA010995C80101966D2DD6
:100A8000F70109951F910F91FF90EF90DF90089566
:100A90000CD0EBC0E3D040F0DAD030F021F45F3F6F
:100AA00019F0CCC0511115C1CFC0F0D098F39923E3
:100AB000C9F35523B1F3951B550BBB27AA27621722
:100AC0007307840738F09F5F5F4F220F331F441F67
:100AD000AA1FA9F333D00E2E3AF0E0E830D091509F
:100AE0005040E695001CCAF729D0FE2F27D0660F8C
:100AF000771F881FBB1F261737074807AB07B0E8CB
:100B000009F0BB0B802DBF01FF2793585F4F2AF0E0
:100B10009E3F510568F092C0DCC05F3FECF3983E09
:100B2000DCF3869577956795B795F7959F5FC9F73D
:100B3000880F911D9695879597F90895E1E0660FC6
:100B4000771F881FBB1F621773078407BA0720F03F
:100B5000621B730B840BBA0BEE1F88F7E0950895A8
:100B600004D06894B111B5C0089598D088F09F570B
:100B700090F0B92F9927B751A0F0D1F0660F771FE9
:100B8000881F991F1AF0BA95C9F712C0B13081F0C9
:100B90009FD0B1E008959CC0672F782F8827B85F59
:100BA00039F0B93FCCF3869577956795B395D9F72A
:100BB0003EF490958095709561957F4F8F4F9F4F34
:100BC0000895E89409C097FB3EF490958095709540
:100BD00061957F4F8F4F9F4F9923A9F0F92F96E989
:100BE000BB279395F695879577956795B795F111FE
:100BF000F8CFFAF4BB0F11F460FF1BC06F5F7F4F9B
:100C00008F4F9F4F16C0882311F096E911C07723AC
:100C100021F09EE8872F762F05C0662371F096E8B5
:100C2000862F70E060E02AF09A95660F771F881F84
:100C3000DAF7880F9695879597F9089597F99F6742
:100C400080E870E060E008959FEF80EC0895002454
:100C50000A941616170618060906089500240A9421
:100C600012161306140605060895092E0394000CA7
:100C700011F4882352F0BB0F40F4BF2B11F460FF36
:100C800004C06F5F7F4F8F4F9F4F089557FD90585F
:100C9000440F551F59F05F3F71F04795880F97FB40
:100CA000991F61F09F3F79F08795089512161306FA
:100CB0001406551FF2CF4695F1DF08C01616170629
:100CC0001806991FF1CF869571056105089408955E
:100CD000E894BB2766277727CB0197F90895991BDE
:100CE00079E004C0991F961708F0961B881F7A9523
:100CF000C9F78095089597FB092E07260AD077FD3E
:100D000004D027D006D000201AF4709561957F4F4B
:100D10000895F6F7909581959F4F089597FB092EBA
:100D200005260ED057FD04D028D00AD0001C38F478
:100D300050954095309521953F4F4F4F5F4F089507
:100D4000F6F790958095709561957F4F8F4F9F4FE7
:100D50000895AA1BBB1B51E107C0AA1FBB1FA61702
:100D6000B70710F0A61BB70B881F991F5A95A9F754
:100D700080959095BC01CD010895A1E21A2EAA1B81
:100D8000BB1BFD010DC0AA1FBB1FEE1FFF1FA2173B
:100D9000B307E407F50720F0A21BB30BE40BF50B38
:100DA000661F771F881F991F1A9469F760957095C1
:100DB000809590959B01AC01BD01CF010895F894F9
:020DC000FFCF63
:100DC200F0204550492D53202D3E204A657469205C
:100DD20020204550492D5465616D20323030392034
:100DE2002000000000000000004D6561737572650F
:100DF2004F7253657474696E6720204D6561737517
:100E020072652020202020203E000000000000000B
:100E1200005370616E6E756E672020205374726F7E
:100E22006D2031302E30562020202031322E30419C
:100E32002000000000000000005370616E6E756EAD
:100E42006720202056657262722031302E30562083
:100E52002020313230306D41680000000000000077
:100E6200004D6561737572654F7253657474696E76
:100E720067202053657474696E672020202020202B
:100E820020000000000000000055736564205365D7
:100E92006E736F722020202020203C2020202020F2
:100EA20020202020202020203E0000000000000002
:100EB200004F66667365742053656E736F722020EF
:100EC20020203C2020202020202020202020202004
:100ED2003E000000000000000000000000000000D2
:100EE2000000000000000000000000000000000000
:100EF20000000000000000000000000000000000F0
:100F020000000000000000000000000000000000DF
:100F120000000000000000000000000000000000CF
:100F220000000000000000000000000000000000BF
:100F320000000000000000000000000000000000AF
:100F4200000000000000000000000000000000009F
:020F5200000598
:00000001FF
